:020000020000FC
:100000001FC028C339C351C351C351C38CC357C385
:100010005AC35AC353C34FC34FC34FC349C349C342
:1000200049C382C352C379C379C37FC37BC379C336
:040030007DC37DC34C
:10004000F894B1E0A0E0D3E0C0E000E00D93BD176C
:10005000E9F7AC17D9F712E00EEF1EBF0DBF00E8AD
:1000600010E0009361001093610007E005B90CEE09
:1000700004B900E408B90FE307B900E00BB902EFD7
:100080000AB900E00093640000E005BF03E00CBB88
:1000900007E005BB00E004BD04E005BD00E006BDCF
:1000A0000FEF07BD0FEF08BD00E003BD00E00093B8
:1000B000800000E00093810000E00093820010E0E7
:1000C00000E0109385000093840010E000E010939E
:1000D00089000093880010E000E010938B000093EB
:1000E0008A0017E001EA109387000093860000E180
:1000F00007BB02E00093B00007E00093B10000E00E
:100100000093B20000E90093B30000E00093B40054
:1001100000E00093B60000E000937C0000E0009354
:100120007A0000E000937B0000E000937E0010E086
:100130000FE21093C5000093C40000E20093C000DA
:1001400008E90093C10006E00093C20001E50CBD80
:1001500000E00DBD0CE00093B80000E00093B90092
:1001600000E70894001F0093BA0000E00093BC0071
:1001700000E80093300000E000937F0004E000936B
:100180006900A89508E10093600008E20093600010
:1001900000E00093680000E000936B0000E0009333
:1001A0006C0000E000936D0001E00DBB00E00093E7
:1001B0006E0000E000936F0002E0009370000BE21D
:1001C000802E902E00E0302E202E03E0702E08EEC0
:1001D000602ED1E0C0E290E007E000931B0003E056
:1001E0000CBB07E005BB07E20093160007E0009395
:1001F000170080E026D5302E81E023D5202E3FE168
:100200002AEF7DD4712E602E172D062D33E028EEB7
:10021000021B130B20F003E0702E08EE602E132D4E
:10022000022D372D262D021B130B18F000E0302E67
:10023000202E3FE12CEF63D4003011F0926002C019
:100240009D7F00C03FE12EEF5AD4003029F094602A
:100250000DB302600DBB02C09B7F00C00FEFFBD44B
:100260007894A89595FF01C07BC190FFFACF9E7F3F
:1002700092FF08C0092D023308F074C0043208F45C
:10028000F0C006C003B101FF6DC000FFEAC000C0AE
:10029000532C422C352D242D32D4103130F4B12F73
:1002A000A02F409A1197F1F7409834E020E0240DF8
:1002B000351D25D4103130F4B12FA02F419A11975C
:1002C000F1F7419838E020E0240D351D18D41031A5
:1002D00030F4B12FA02F429A1197F1F742983CE0E9
:1002E00020E0240D351D0BD4103130F4B12FA02F98
:1002F000439A1197F1F7439830E120E0240D351D22
:10030000FED3103130F4B12FA02F449A1197F1F79A
:10031000449834E120E0240D351DF1D3103130F440
:10032000B12FA02F459A1197F1F7459838E120E0B9
:10033000240D351DE4D3103130F4B12FA02F5E9A77
:100340001197F1F75E983CE120E0240D351DD7D3DD
:10035000103130F4B12FA02F5F9A1197F1F75F9809
:1003600000C077C1532C422C352D242DC8D3103119
:1003700030F4B12FA02F409A1197F1F7409834E054
:1003800020E0240D351DBBD3103130F4B12FA02F48
:10039000419A1197F1F7419838E020E0240D351D7E
:1003A000AED3103130F4B12FA02F429A1197F1F74C
:1003B00042983CE020E0240D351DA1D3103130F4EB
:1003C000B12FA02F439A1197F1F7439830E120E025
:1003D000240D351D94D3103130F4B12FA02F449A41
:1003E0001197F1F7449834E120E0240D351D87D3AF
:1003F000103130F4B12FA02F459A1197F1F745989D
:1004000038E120E0240D351D7AD3103130F4B12FBE
:10041000A02F5E9A1197F1F75E983CE120E0240D41
:10042000351D6DD3103130F4B12FA02F5F9A119785
:10043000F1F75F98172D062D332D222D201B310B40
:1004400040F091FD01C00CC000E0302E00E0202EF5
:1004500007C002E010E0F894200E311E789400C02E
:10046000F8C0532C422C352D242D49D3103130F4B3
:10047000B12FA02F409A1197F1F7409834E020E077
:10048000240D351D3CD3103130F4B12FA02F419AEB
:100490001197F1F7419838E020E0240D351D2FD356
:1004A000103130F4B12FA02F429A1197F1F74298F2
:1004B0003CE020E0240D351D22D3103130F4B12F63
:1004C000A02F439A1197F1F7439830E120E0240DD3
:1004D000351D15D3103130F4B12FA02F449A119748
:1004E000F1F7449834E120E0240D351D08D3103194
:1004F00030F4B12FA02F459A1197F1F7459838E1C4
:1005000020E0240D351DFBD2103130F4B12FA02F87
:100510005E9A1197F1F75E983CE120E0F894240D83
:10052000351D7894ECD2103130F4B12FA02F5F9AA2
:100530001197F1F75F9810E000E0332D222D021B98
:10054000130B30F091FD01C00AC0372C262C07C0D8
:1005500002E010E0F894201A310A789400C079C0C3
:10056000009170000D7F009370000DB30D7F0DBBE7
:10057000F0E0E0E050E0A89596FFFDCF9F7B97FF6D
:1005800001C003C0B1E0A0E202C0B1E0A0E853D2D4
:1005900001E061D32A9802E00EBD2DB527FFFDCF03
:1005A0002EB5FEBD2DB527FFFDCF2EB5EEBD2DB569
:1005B00027FFFDCF2EB540E13D912D911D910D916D
:1005C000CCD01EBD2DB527FFFDCF2EB50EBD2DB550
:1005D00027FFFDCF2EB50D910D914A9569F72A9A07
:1005E000B09601E038D35A9531F600E0302E00E0A5
:1005F000202E75EA80E0032D15D381E0022D12D361
:1006000070E003E50093000105E70093010103E6B4
:100610000093020103E60093030105E60093040141
:1006200003E70093050103E70093060107E080D08C
:100630009F7D80E00091700002600093700092FF47
:1006400003C00DB302600DBBF894D1E0C0E2789412
:10065000F7CC07CEFFB60F9375EA80E0032DE2D208
:1006600081E0022DDFD270E0A89505E0F4D24A9B2C
:10067000FBCF0F91FFBE1895FFB60F934B9B02C0A7
:1006800086B410C006B508190E3060F0091528F4BC
:10069000092D073108F09A9405C0092D0F3308F48D
:1006A000939400C00F91FFBE189518951895189552
:1006B0001895189518951895189518951895FFB6CA
:1006C0009160FFBE189518951895FFB60F9300918D
:1006D000C600CF3F08F409930A3081F4009120014D
:1006E0000B3261F4009121010B3241F4009122019F
:1006F0000B3221F49062D1E0C0E20CC0C03819F492
:100700009F77906407C0C03E29F4D1E0C0E29068B2
:10071000906400C00F91FFBE189518951895189514
:100720001895189518951895189518951895189561
:100730001F932F93EF93FF93202FF1E0E0E01091B0
:10074000C00015FFFCCF01910093C6002A95B9F7B0
:10075000FF91EF912F911F9108950F921F922F9269
:100760003F924F935F93AF93BF9340E050E030537D
:10077000205310530053332E222E112E002E10E042
:10078000032D33E028EE0E9480048894401F511FFF
:1007900010E0022D30E024E60E9480048894401F7F
:1007A000511F10E0012D30E02AE00E94800488945F
:1007B000401F511F10E0002D8894401F511F152F1E
:1007C000042FBF91AF915F914F913F902F901F9059
:1007D0000F9008956F937F938F93AF93712F602F36
:1007E00040E030E020E010E000E08894A7E280E103
:1007F000680B7A0B439577FFF8CF8894681F7A1FB0
:100800004A958894A3E088EE680B7A0B339577FFBE
:10081000F8CF8894681F7A1F3A958894A0E084E600
:10082000680B7A0B239577FFF8CF8894681F7A1F9F
:100830002A958894A0E08AE0680B7A0B139577FFDD
:10084000F8CF8894681F7A1F1A95062F50E3450F3A
:10085000350F250F150F050FAF918F917F916F9178
:1008600008953F9334E620E02395031BE8F72A958B
:10087000030F3AE010E01395031BE8F71A95030FF6
:1008800030E3230F130F030F3F9108950F921F9230
:100890002F923F924F935F93AF93BF9340E050E00E
:1008A0003053205310530053332E222E112E002E7E
:1008B00010E0032D33E028EE23D08894401F511F11
:1008C00010E0022D30E024E61BD08894401F511F19
:1008D00010E0012D30E02AE013D08894401F511F12
:1008E00010E0002D8894401F511F152F042FBF9139
:1008F000AF915F914F913F902F901F900F9008956F
:100900004F935F936F93412F532F452B47FF08C0A1
:10091000412F532F452347FD05C017FD11C022C0AD
:1009200037D032C01095009541E0040F40E0141F0D
:100930003095209541E0240F40E0341F29D024C099
:100940001095009541E0040F40E0141F21D0309530
:1009500020951095009541E0040F40E0141F241FDE
:10096000341F12C03095209541E0240F40E0341F21
:100970000FD0309520951095009541E0040F40E090
:10098000141F241F341F00C06F915F914F91089571
:10099000551B441B61E110F4400F511F57954795BB
:1009A000379527956A95B9F75F934F933F932F93A8
:1009B0000F911F912F913F910895AF93BF93CF93C4
:1009C000DF93B12FA02FD32FC22F0D9109934A95FA
:1009D000E1F7DF91CF91BF91AF91089505E007D086
:1009E000089505E304D0089503E301D008951F930B
:1009F0002A9815E01EBD1DB517FFFDCF1EB510E0EE
:100A00001EBD1DB517FFFDCF0EB52A9A1F91089583
:100A10000F932A9805E00EBD0DB507FFFDCFA895F1
:100A200000E00EBD0DB507FFFDCF0EB500FDF7CF01
:100A30002A9A0F9108950F932A9806E00EBD0DB5DE
:100A400007FFFDCF2A9A0F9108950F932A9804E08B
:100A50000EBD0DB507FFFDCF0EB52A9A0F91089573
:100A60000F932A9806E60EBD0DB507FFFDCF0EB514
:100A70002A9A0F9108950F932A9809E90EBD0DB592
:100A800007FFFDCF0EB52A9A0F9108955F932A981C
:100A900052E05EBD5DB557FFFDCF5EB52EBD5DB5C5
:100AA00057FFFDCF5EB51EBD5DB557FFFDCF5EB5EF
:100AB0000EBD5DB557FFFDCF5EB52A9A5F910895D3
:100AC0005F932A9852E05EBD5DB557FFFDCF5EB5DE
:100AD0003EBD5DB557FFFDCF5EB52EBD5DB557FF81
:100AE000FDCF5EB51EBD5DB557FFFDCF5EB50EBD3A
:100AF0005DB557FFFDCF5EB52A9A5F9108955F936C
:100B00002A9853E05EBD5DB557FFFDCF3EBD5DB594
:100B100057FFFDCF2EBD5DB557FFFDCF5FEF5EBD2B
:100B20005DB557FFFDCF1EB55FEF5EBD5DB557FFED
:100B3000FDCF0EB52A9A5F9108950F932A9807EC7E
:100B40000EBD0DB507FFFDCF0EB52A9A0F91089582
:100B50003F932A9838ED3EBD3DB537FFFDCF3EB5FA
:100B600030E03EBD3DB537FFFDCF3EB530E03EBD88
:100B70003DB537FFFDCF3EB530E03EBD3DB537FF5B
:100B8000FDCF3EB52A9A3F9108953F932A9831E0D0
:100B90003EBD3DB537FFFDCF3EB50EBD3DB537FF80
:100BA000FDCF3EB51EBD3DB537FFFDCF3EB52EBDD9
:100BB0003DB537FFFDCF3EB52A9A3F9108952F925C
:100BC0003F924F921F932A984090CA043090CB04D2
:100BD0002090CC0413E01EBD1DB517FFFDCF4EBC09
:100BE0001DB517FFFDCF3EBC1DB517FFFDCF2EBCB9
:100BF0001DB517FFFDCF1FEF1EBD1DB517FFFDCFA4
:100C00000EB5089410E0211E311E411E4092CA0408
:100C10003092CB042092CC042A9A1F914F903F909F
:100C20002F9008951F93F999FECF10E01FBB10E09D
:100C300012BD81BD00BD753A11F4FA9AF99A1F915F
:100C400008951F93F999FECF10E012BD81BDF89A67
:100C500000B51F9108951F932F932AE01AEF1A955C
:100C6000F1F72A95D9F70A95C1F72F911F910895A9
:00000001FF
